:020000040000FA
:1000000000EF04F01200FFFF04EF04F01200FFFF06
:10001000FFFFFFFFFFFFFFFF0CEF04F01200FFFFE9
:10002000FFFFFFFFFFFFFFFFFFFF0100E2070000F0
:100030007E000000020000000001776B1E0E716E52
:100040000401400E096F200E0A6F040E0B6F880E1C
:10005000086F0401200E0E6F040E0F6F400E0C6F20
:100060001200550EA76EAA0EA76EA68212000401FA
:10007000140E226F010E236F12000001756B5CD904
:100080000AE267D90800F5CF76F000014ED976C0B4
:10009000EFFF752BF4D7F86A1200F00E0401221757
:1000A000840EA66E0001756B47D90AE24AD90F0E7D
:1000B000000175150F0801E1D4DF0001752BF4D79D
:1000C0001200940EA66E0001756B36D911E27551BF
:1000D000006E016A060ED89000360136E804FBE196
:1000E000026A01BE026812D9BCDF0001752BEDD790
:1000F000F86A1200A66A0001756B1ED90BE20401B2
:10010000225100017525A96EA6800FD9A8CFEFFF57
:10011000752BF3D712000001756B0ED910E20401A4
:10012000225100017525A96E00D9EF50A86E040E6A
:10013000A66E97DFA6B2FED70001752BEED7120090
:10014000C40EA66E0001756BF7D805E2FAD889DFF8
:100150000001752BF9D7F86A120097D8060E000136
:100160007A5D03E36D50020B01E08ED0000177054C
:1001700011E104010CBF0DD00401400E096F400EC7
:10018000040108170401087D880E0401081300010A
:10019000776B7AD0040108BF77D00001756B04013A
:1001A0002051320A45E0CD0A34E0F80A2DE0020A77
:1001B00026E0010A1FE0070A18E0010A11E0030A1D
:1001C0000AE0070A08E0060A01E04DD050DF00010E
:1001D000040E756F49D051DF050E0001752744D01C
:1001E0005CDF0001010E756F3FD06BDF0001010E77
:1001F000756F3AD07FDF050E0001752735D08BDF94
:100200000001010E756F30D09BDF0001010E756F8C
:100210002BD06D960001786B796B00017807000E8A
:10022000795B00017851791101E0F7D7FF001CD00C
:10023000030E0401215D09E104012251E8B08C8420
:10024000E8A08C940001010E756F040E0401215D7D
:1002500009E104012251E8B08C86E8A08C960001E7
:10026000010E756F01D000D00001010E776F000103
:1002700075510AE075C00DF4400E04010C1704011D
:100280000C7D880E04010C13120000017E517F11B9
:1002900004E1200E7E6F4E0E7F6F7E07000E7F5BA7
:1002A0006DA208D07E517F1130E18C708C50010B13
:1002B00013E128D000017A5102E18C9023D07A0515
:1002C00002E18C8009D0020E7A5D02E18C801AD0A6
:1002D000030E7A5D03E18C908C821200050E7A5D2C
:1002E00006E100017E517F1110E18C700BD0060EEB
:1002F0007A5D0BE100017E517F1107E18C708C501B
:10030000010B02E08C9212008C8212000401225137
:100310000024F36E23510120F46E24510220F86E64
:10032000F4CFF7FFF3CFF6FF12007551EA6A250FFD
:10033000E96E040EEA221200040121510001755DEC
:100340001200F3DFEFCF03F004D803C0F5FF0C0079
:10035000120075C000F0016A026A86EF01F06C506D
:100360000BE1040100513C0BE842E8420D0802E1B8
:10037000C1EF01F0CAEF01F0040E6C5C01E119D885
:1003800012000001606B616B666B676B95EC02F0AD
:100390004CEF02F0020E0001605D09E15CD804013F
:1003A00000BD02D0C80E01D0880E006F120085EF8C
:1003B00002F0040E00017A5D09E112C46EFF6E5076
:1003C000000802E2050E01D0030E7A6F00016005FD
:1003D00009E10AD8040104BD02D0C80E01D0880E7C
:1003E000046F120085EF02F00001080E665D000E3A
:1003F000675903E266C069F002D0080E696F69C0F0
:1004000005F46951006E016A0050665F0150675B38
:10041000180E646F040E656F69511CE000017BA328
:1004200007D062C0F6FF63C0F7FF0800F55005D0A3
:1004300062C0E9FF63C0EAFFEF5064C0E9FF65C036
:10044000EAFFEF6E0001622B000E6323642B65232D
:100450006907E2D7120001C46AF000016A516625FB
:10046000666F000E6721676F180E626F040E636F70
:100470006A5111E062C0E9FF63C0EAFFEF5064C057
:10048000E9FF65C0EAFFEF6E642B000E6523622B67
:1004900063236A07EDD712006D980001615105E1F1
:1004A0003CD8840E006F04011DD0040110AF1CD095
:1004B000000166510401165D0001675104011759DE
:1004C00004E216C466F017C467F08EDF0001010E67
:1004D000606F23D8800E006F0401180E066F040EA3
:1004E000076FC80E046F12000001020E606F040156
:1004F000056BC80E046F0401080E016F180E026F21
:10050000040E036FC80E006F12000001606B05D867
:100510008C0E006F0401046B12000401080E016FC1
:10052000100E026F040E036F120004011051600BD5
:10053000E842E842E842E842E842000901E01200ED
:100540001151080A39E0010A35E00F0A0AE0030AEE
:1005500001E012000001010E616F0001040E7A6FCC
:1005600012000001010E616F0401130507E1000193
:100570004C0E626F070E636F120E13D0020E135DE6
:1005800007E100015E0E626F070E636F200E09D057
:10059000030E135D0AE100017E0E626F070E636FAA
:1005A000040E0001666F676B02D00001616B0001F1
:1005B0007B831200EAEF02F00001010E616F00017F
:1005C0007C0E626F000E636F00017B930001010ED1
:1005D000666F12000001010E616F12C47CF004010D
:1005E000125104E10001050E7A6F12000001060E9F
:1005F0007A6F1CEF00F0080E6D6E6DBAFED7686A58
:10060000110E696E0001020E7A6F12006850040B21
:1006100009E06950040B06E06D92699468A402D069
:100620006894FCD76850010B04E06950010B01E0AD
:1006300025D86850100B0AE06950100B07E0698458
:1006400068986D82A19AA08A0300A19A6850200B35
:1006500006E06950200B03E070B07090689A030EBA
:1006600000017A5D01E209D06850080B06E069508C
:10067000080B03E0AFEC01F068961200686A7B0E8D
:10068000696E6E6A160E706E68A608D068960000D5
:1006900000000000000000000000F6D76D9885EC17
:1006A00002F000017C6B0001030E7A6F12002A0E2B
:1006B000F66E000EF76E000EF86E00010900F550A0
:1006C000706F0900F550716F03E1706701D03DD084
:1006D0000900F5506B6F0900F5506C6F0900F5507B
:1006E0006D6F09000900F550E96E0900F550EA6EDA
:1006F000090009000900F5506E6F0900F5506F6F91
:1007000009000900F6CF72F0F7CF73F0F8CF74F05C
:100710006BC0F6FF6CC0F7FF6DC0F8FF00016E53B1
:1007200002E16F5307E00900F550EE6E6E07F8E244
:100730006F07F9D772C0F6FF73C0F7FF74C0F8FFF8
:1007400000017007000E715BBFD71200120100029A
:1007500000000008D8040B0001000000000109029D
:1007600020000101008032090400000200000000A6
:100770000705010240000007058102400000040354
:100780000904C1CF80F00F0EC112819A939A81B8EB
:1007900004D080C0C1FF00EF04F0F00E8C16F00E04
:1007A0009516140E6F6EFBEC02F006EC03F0ADEC48
:1007B00000F0FBD7120013EE00F023EE00F0F86A11
:1007C000059C57EC03F0F0EC03F0C1EC03F0FBD711
:1007D000120000EE00F00F0EEE6AEA62FDD7120082
:1007E00012000000FFFFFFFFFFFFFFFFFFFFFFFF03
:1007F000FFFFFFFFFFFFFFFFFFFFFFFFFFFFFFFF09
:10080000CDEF14F01200FFFF1200FFFFFFFFFFFF0C
:10081000FFFFFFFFFFFFFFFF1200FFFFFFFFFFFFD4
:10082000FFFFFFFFFFFFFFFFFFFF0100B8290000F0
:100830001A0100000200000001010B6B086B166B2F
:100840001200D9CFE6FFE1CFD9FFE150FB0FE66EF2
:10085000FF0EDA20E66E4FEC0DF0E552E552FB0E8E
:10086000DBCF17F0FC0EDBCF18F0FD0EDBCF19F05D
:10087000FE0EDBCF1AF017C010F018C011F019C02F
:1008800012F01AC013F0E552E7CFD9FF1200080E9C
:10089000E66E40EC0EF0E5520C0EE66E010EE66ED2
:1008A0004FEC0DF0E552E5521200D9CFE6FFE1CF53
:1008B000D9FF040EE1260A0EE66E40EC0EF0E5527A
:1008C000E66AC00EE66E040EE66EE66ABADFE55230
:1008D000E552E552E55210C0DEFF11C0DEFF12C046
:1008E000DEFF13C0DDFFDD52DD52020EDBCF09F16A
:1008F000030EDBAE03D00101010E0B6F080E176E65
:10090000186A196A1A6AD9CFE9FFDACFEAFFEE50FE
:100910001716EE501816EE501916EE501A161750FC
:10092000181019101A1004E00101010E0A6F02D00C
:1009300001010A6B040EE15C02E2E16AE552E16E3C
:10094000E552E7CFD9FF12000A0EE66E40EC0EF03A
:10095000E552E66AD00EE66E040EE66EE66A71DFD8
:10096000E552E552E552E5521200D9CFE6FFE1CF5C
:10097000D9FF040EE126090EE66E40EC0EF0E552BA
:10098000D950FB0FE96EFF0EDA20EA6EEECFE6FFDC
:10099000EECFE6FFEECFE6FFEFCFE6FF52DFE55208
:1009A000E552E552E55210C0DEFF11C0DEFF12C075
:1009B000DEFF13C0DDFFDD52DD52DECF10F0DECFF3
:1009C00011F0DECF12F0DDCF13F0DD52DD52040E58
:1009D000E15C02E2E16AE552E16EE552E7CFD9FF60
:1009E0001200D9CFE6FF020EE1260101165102E006
:1009F000086902D0010E166F020EE15C02E2E16AA4
:100A0000E552E16EE552E7CFD9FF1200D9CFE6FFFC
:100A1000E1CFD9FFE6520CC117F00DC118F00EC19D
:100A200019F00FC11AF0040E185E200E195AFF0EAD
:100A30001A5A020ED8901A32193218321732E806B2
:100A4000F9E11750DF6E010109A724D0E66AE66AD2
:100A5000E66AE66A8ADFE552E552E552E55210C0E1
:100A600017F011C018F012C019F013C01AF0DF50BF
:100A7000040DF3CFE9FFF4CFEAFF000EE926060EDE
:100A8000EA2210C0EEFF18C0EEFF19C0EEFF1AC038
:100A9000EEFF17D0DF50040DF3CFE9FFF4CFEAFFEC
:100AA000000EE926060EEA22EECFE6FFEECFE6FFC5
:100AB000EECFE6FFEFCFE6FF58DFE552E552E55215
:100AC000E5520A0EE66E40EC0EF0E552E66AC00E04
:100AD000E66EE66AE66AB5DEE552E552E552E552B3
:100AE000E552E552E7CFD9FF1200D9CFE6FFE1CFBB
:100AF000D9FFE65201010C51E840E8403F0B010BE1
:100B0000DF6EDF50040DF3CFF6FFF4CFF7FF1A0EC0
:100B1000F626290EF7220900F5CFE6FF0900F5CFEA
:100B2000E6FF0900F5CFE6FF0800F5CFE6FF1DDF81
:100B3000E552E552E552E5520A0EE66E40EC0EF043
:100B4000E552E66AC00EE66EE66AE66A7ADEE552CD
:100B5000E552E552E552E552E552E7CFD9FF1200E2
:100B6000010108510B0A01E122D3010A01E1F8D287
:100B7000030A01E1CDD1010A01E1B3D10F0A01E17C
:100B8000AAD1010A01E129D1030A01E1B0D0060A84
:100B900033E0070A31E0060A10E0030A05E0010A23
:100BA00001E012008B9407D080DE01010B5101E1BE
:100BB00005D3020E086F0B6B120077DE010109A549
:100BC000FDD28B8464DE01010C510CE1040E0D1981
:100BD00009E1200E0E1906E1E8680F1903E1030E82
:100BE000086F01D082DF0CC110F10DC111F10EC1EF
:100BF00012F10FC113F11200165101E1DFD2000111
:100C0000A451020B03E1A451010B02E001017AD1CE
:100C10000101186B196B040E19AF02D0D89003D0E4
:100C2000185D000E195949E218C1F6FF19C1F7FF06
:100C3000030ED890F636F736E806FBE1220EF626CC
:100C4000290EF7220900F5CF17F00900F5CF18F0AB
:100C50000900F5CF19F00900F5CF1AF00900F5CF1A
:100C60001BF00900F5CF1CF00900F5CF1DF00800BE
:100C7000F5CF1EF018C1E9FF19C1EAFF030ED890A5
:100C8000E936EA36E806FBE1820EE926000EEA22A2
:100C900017C0EEFF18C0EEFF19C0EEFF1AC0EEFF3E
:100CA0001BC0EEFF1CC0EEFF1DC0EEFF1EC0EEFF1E
:100CB0000101182B000E1923AED70001010EA36FFE
:100CC0000001A4830101070E086F166BABC000F78B
:100CD000ACC001F7ADC002F7AEC003F7AFC004F778
:100CE000B0C005F7B1C006F7B2C007F7120017058C
:100CF000080DF3CFE9FFF4CFEAFF820EE926000EDC
:100D0000EA22020EE926000EEA22EF50020801E074
:100D100055D217052EE1186B196B100E19AF02D0C2
:100D2000D89003D0185D000E19591EE218C118F0B2
:100D300019C119F0D89018361936D89018361936C6
:100D4000000E1826050E192218C0E6FF19C0E6FF8E
:100D5000FBEC0BF0E552E552176EE834E7E30101D6
:100D6000182B000E1923D9D70001846B0101020E44
:100D70002ED0100E186F196B200E19AF02D0D8901C
:100D800003D0185D000E19591EE218C118F019C1E0
:100D900019F0D89018361936D89018361936000E32
:100DA0001826050E192218C0E6FF19C0E6FFFBEC55
:100DB0000BF0E552E552176EE834E7E30101182B1A
:100DC000000E1923D9D700018C6B0101010E176F9A
:100DD0000001A4B3F3D1010199D01705080DF3CF99
:100DE000E9FFF4CFEAFF620EE926000EEA22020EC6
:100DF000E926000EEA22EF50020801E0DFD10101EE
:100E00001A2B000E1B23010117052EE1186B196B1D
:100E1000100E19AF02D0D89003D0185D000E1959EA
:100E20001EE218C118F019C119F0D89018361936F9
:100E3000D89018361936000E1826050E192218C03B
:100E4000E6FF19C0E6FFB5EC0CF0E552E552176E6F
:100E5000E834E7E30101182B000E1923D9D700016C
:100E6000646B0101020E2ED0100E186F196B200E4C
:100E700019AF02D0D89003D0185D000E19591EE2A8
:100E800018C118F019C119F0D89018361936D89031
:100E900018361936000E1826050E192218C0E6FF5E
:100EA00019C0E6FFB5EC0CF0E552E552176EE834D8
:100EB000E7E30101182B000E1923D9D700016C6B51
:100EC0000101010E176F1407000E155B1451151167
:100ED00001E074D11BD00001A4B370D10101080E50
:100EE0006BD1E3DC010109A569D1D1DC01010C5111
:100EF00008E1040E0D1905E1200E0E1902E1E86863
:100F00000F1902E00869120081DD0101090E54D1B8
:100F1000CCDC010109A51ED1BADC01010C510BE1A9
:100F2000040E0D1908E1200E0E1905E1E8680F19ED
:100F300002E10A0E41D10C5101E0FDD00D5101E05A
:100F4000FAD0200E0E1901E0F6D0E8680F1901E082
:100F5000F2D0010E176F09A778D0186B196B020E2B
:100F600019AF02D0D89003D0185D000E195949E28C
:100F700018C1F6FF19C1F7FF030ED890F636F73601
:100F8000E806FBE14A0EF626290EF7220900F5CF06
:100F900017F00900F5CF18F00900F5CF19F0090096
:100FA000F5CF1AF00900F5CF1BF00900F5CF1CF0C2
:100FB0000900F5CF1DF00800F5CF1EF018C1E9FFBC
:100FC00019C1EAFF030ED890E936EA36E806FBE1DC
:100FD000620EE926000EEA2217C0EEFF18C0EEFFEF
:100FE00019C0EEFF1AC0EEFF1BC0EEFF1CC0EEFFE3
:100FF0001DC0EEFF1EC0EEFF0101182B000E1923CD
:10100000AED704C717F005C718F006C719F007C711
:101010001AF0040ED8901A32193218321732E80634
:10102000F9E117C014F118C015F117C070F018C01D
:1010300071F00001D890713370330001010EA26F7E
:101040000001A4810101060E6FD0186B196B020E0E
:1010500019AF02D0D89003D0185D000E195949E29B
:1010600018C1F6FF19C1F7FF030ED890F636F73610
:10107000E806FBE15A0EF626290EF7220900F5CF05
:1010800017F00900F5CF18F00900F5CF19F00900A5
:10109000F5CF1AF00900F5CF1BF00900F5CF1CF0D1
:1010A0000900F5CF1DF00800F5CF1EF018C1E9FFCB
:1010B00019C1EAFF030ED890E936EA36E806FBE1EB
:1010C000820EE926000EEA2217C0EEFF18C0EEFFDE
:1010D00019C0EEFF1AC0EEFF1BC0EEFF1CC0EEFFF2
:1010E0001DC0EEFF1EC0EEFF0101182B000E1923DC
:1010F000AED704C717F005C718F006C719F007C721
:101100001AF0050ED8901A32193218321732E80642
:10111000F9E117C090F018C091F00001010EA36F23
:101120000001A4830101050E086F0E0EE66E40EC6F
:101130000EF0E55212000C510BE1020E0D1908E100
:10114000200E0E1905E1E8680F1902E1020E34D0F5
:1011500006EF05F00A5132E1020E086F8B9412007F
:101160000001A4B124D0420EF66E290EF76E0900DC
:10117000F5CF62F00900F5CF63F00900F5CF64F018
:101180000900F5CF65F00900F5CF66F00900F5CF4D
:1011900067F00900F5CF68F00800F5CF69F00001AD
:1011A000010EA26F0001A48101010B0E086F000166
:1011B000A4B104D00101040E086F12001200D9CFAF
:1011C000E6FFE1CFD9FFFE0EDB50A96EFD0EDB502E
:1011D000A86E040EA66E550EA76EAA0EA76EA68266
:1011E000A6B2FED7E552E7CFD9FF1200026802503F
:1011F00002E00206FCD71200D9CFE6FFE1CFD9FF0B
:10120000040EE126DE6ADE6A020EDE6EDD6ADD5263
:10121000DD52D9CFE9FFDACFEAFFEECF17F0EECFFC
:1012200018F0EECF19F0EFCF1AF017501810191070
:101230001A100AE0D9CFE9FFDACFEAFFEE06000E76
:10124000EE5AEE5AEE5AE5D7040EE15C02E2E16A8C
:10125000E552E16EE552E7CFD9FF120081A002D03E
:10126000008401D000948A92939000A802D08A80D2
:1012700001D08A908A828A9200A602D08A8001D008
:101280008A908A828A9293808A828A928A821200C3
:1012900000A802D0898601D0899600A602D0898450
:1012A00001D0899480A002D0008401D0009489826A
:1012B0008992120000A002D048EF09F02EEF09F049
:1012C00000965AEF09F09382938012008A928A90D6
:1012D0009392939012009480120094901200928640
:1012E00092809284928200821200899289968994D7
:1012F0009296928092949292009212000086026AD4
:10130000050E025C03E2D6DF022AFAD760EF09F08D
:101310000086D0DF0096CEDF5AEF09F0A8C005F0B6
:10132000200E055C0BE1020E076EA90EE66E000EA4
:10133000E66E4FEC0DF0E552E5523CD0E9DF010ED0
:10134000086E046A0550045C28E2070E041411E1DB
:101350000850EA6AA70FE96E000EEA2203C0EFFF09
:10136000082A0850EA6AA70FE96E000EEA22EF5039
:10137000036E0504045C01E10086010E031400986D
:10138000E8B0008897DF03407F0B036E00A403D012
:10139000800E0310036E042AD5D705C0A8F00850AC
:1013A000EA6AA70FE96E000EEA2203C0EFFF00868B
:1013B00081DF00965AEF09F000867CDF010E086E8F
:1013C000A7DFA8C005F0046A0550045C28E2070EF8
:1013D000041411E10850EA6AA70FE96E000EEA2230
:1013E00003C0EFFF082A0850EA6AA70FE96E000E53
:1013F000EA22EF50036E0504045C01E10086010E51
:1014000003140098E8B0008855DF03407F0B036E9B
:1014100000A403D0800E0310036E042AD5D705C0A4
:10142000A8F00850EA6AA70FE96E000EEA2203C08E
:10143000EFFF40DF00965AEF09F0D9CFE6FFE1CF8A
:10144000D9FFE65265DF009835DF0050040B01E05C
:10145000010EDF6E0750086E046A200E045C1BE26A
:10146000070E041409E10850EA6AA70FE96E000E9E
:10147000EA22EF50036E082A1F0E045C01E1008689
:10148000010E03140098E8B0008814DF03407F0BBE
:10149000036E042AE2D70EDF00960CDFDF50E55220
:1014A000E552E7CFD9FF1200010E086E046A200E44
:1014B000045C1BE2070E041409E1082A0850EA6ADA
:1014C000A70FE96E000EEA22EF50036E03AE02D0C2
:1014D0008A8001D08A908ADE8A8288DE8A9286DEBD
:1014E00003500324036E042AE2D712000090EEDEBC
:1014F0008B807CDE8B907ADE00014D0EA96F430E4F
:10150000AA6F480EAB6F500EAC6FCEDF6FDE8B80D4
:101510006DDEF4DE0001050EA86F040EA96F4CDF2E
:101520000001050EA86F070EA96F46DF0001080E27
:10153000A86FFC0EA96FF2DE5FDE0001080EA86F37
:10154000A96BECDEFFD7D9CFE6FFE1CFD9FF060EBE
:10155000E126DE6ADE6ADE6ADD6ADD52DD52040EF5
:10156000DB6A050EDB6AD09C066A8A9A939A8B9492
:10157000949442DED08CB3DEA6DEADDE1CEC04F02B
:10158000060EE15C02E2E16AE552E16EE552E7CF68
:10159000D9FF1200060E0001F95D09E36D50020B40
:1015A00001E01200B0EC05F04EEC11F001D8120091
:1015B000D9CFE6FFE1CFD9FFE652400EE66EA70E87
:1015C000E66E000EE66E96EC13F0E552E552E5523B
:1015D000000901E10BD1016A0001A751FE0A01E1F6
:1015E000E8D0FB0A01E1DBD0370A01E1D5D0030ADC
:1015F00001E1CDD0B10A01E1C8D0010A01E1C3D0B7
:10160000AC0A01E1B7D0010A01E1ACD03C0A01E12A
:1016100096D0EF0A01E191D0DD0A01E18CD0030AF6
:1016200001E187D0040A01E182D0010A01E17DD005
:101630000F0A01E178D0010A74E0040A6DE0010AA2
:1016400066E00C0A62E00A0A49E00F0A2EE00E0A80
:1016500015E0080A0CE0200A01E0B7D00001070EEF
:10166000A96F0001020EAA6F040E016EAFD0000137
:10167000A85102E0008001D00090A8D09DDE070EA6
:101680000001A81509E00001A851E840E840E84041
:101690001F0B030F016E08D00001A851E840E8407D
:1016A000E8401F0B020F016E91D00001A951E8B074
:1016B0008984E8A089940001AA51E8B08986E8A04D
:1016C00089960001AB51E8B08982E8A089928050E8
:1016D000010B0001A96F050E016E78D01FDE070E09
:1016E0000001A81509E00001A851E840E840E840E1
:1016F0001F0B030F016E08D00001A851E840E8401D
:10170000E8401F0B020F016E61D0CEDE5FD0A8C093
:1017100006F0020E076E5AD0A8C006F0020E076E41
:1017200055D0D9DD53D0D9DD51D0D9DD4FD0DDDD55
:101730004DD0C9DD4BD0CADD49D0E0DD47D0ABC0CC
:1017400000F1ACC001F1ADC002F1AEC003F1AFC019
:1017500004F1B0C005F1B1C006F1B2C007F1F1EC7F
:1017600004F034D00101086B8B90030E016E08C1A8
:10177000A9F02CD00101010E086F8B80030E016EC1
:1017800008C1A9F023D08A9A21D08A8A1FD0030EDB
:10179000016E08C1A9F01AD0A4EC04F017D0ACC0B7
:1017A000E6FFA9C0E6FF0BDDE552E552010E016E32
:1017B0000DD06D960A6A0B6A0A06000E0B5A0A5083
:1017C0000B1001E0F9D7FF0001D000D001500EE06E
:1017D00004010CBF0BD00150E66EA70EE66E000EA2
:1017E000E66E5DEC13F0E552E552E552E552E55246
:1017F000E7CFD9FF120089848982896A8982899218
:1018000089828992898280300932896AFE0EE3CF0B
:10181000E9FFFF0EE3CFEAFFEE3001E3898689821C
:10182000896AE83001E389868982896AE83001E3C0
:1018300089868982896AE83001E389868982896A92
:10184000E83001E389868982896AE83001E3898684
:101850008982896AE83001E389868982896AE83069
:1018600001E389868982896AEE3001E3898689826B
:10187000896AE83001E389868982896AE83001E370
:1018800089868982896AE83001E389868982896A42
:10189000E83001E389868982896AE83001E3898634
:1018A0008982896AE83001E389868982896AE83019
:1018B00001E389868982896AEE3001E3898689821B
:1018C000896AE83001E389868982896AE83001E320
:1018D00089868982896AE83001E389868982896AF2
:1018E000E83001E389868982896AE83001E38986E4
:1018F0008982896AE83001E389868982896AE830C9
:1019000001E389868982896AEE3001E389868982CA
:10191000896AE83001E389868982896AE83001E3CF
:1019200089868982896AE83001E389868982896AA1
:10193000E83001E389868982896AE83001E3898693
:101940008982896AE83001E389868982896A898483
:10195000E83001E389868982896A8984898289924B
:10196000896A898289920950120089848982896AE8
:101970008982899289828992898280300932896A32
:10198000FE0EE3CFE9FFFF0EE3CFEAFF898280304E
:10199000EF32896A89828030EF32896A89828030A9
:1019A000EF32896A89828030EF32896A8982803099
:1019B000EF32896A89828030EF32896A8982803089
:1019C000EF32896A89828030EE32896A898280307A
:1019D000EF32896A89828030EF32896A8982803069
:1019E000EF32896A89828030EF32896A8982803059
:1019F000EF32896A89828030EF32896A8982803049
:101A0000EF32896A89828030EE32896A8982803039
:101A1000EF32896A89828030EF32896A8982803028
:101A2000EF32896A89828030EF32896A8982803018
:101A3000EF32896A89828030EF32896A8982803008
:101A4000EF32896A89828030EE32896A89828030F9
:101A5000EF32896A89828030EF32896A89828030E8
:101A6000EF32896A89828030EF32896A89828030D8
:101A7000EF32896A89828030EF32896A89828030C8
:101A8000EF32896A898489828030EE32896A89845A
:101A900089828992896A898289920950120089848F
:101AA0008982896A8982899289828992FE0EE3CF2E
:101AB000E9FFFF0EE3CFEAFF00008030EF3201E3E1
:101AC00089868982896A00008030EF3201E3898645
:101AD0008982896A00008030EF3201E38986898239
:101AE000896A00008030EF3201E389868982896A41
:101AF00000008030EF3201E389868982896A000024
:101B00008030EF3201E389868982896A0000803063
:101B1000EF3201E389868982896A00008030EE32E3
:101B200001E389868982896A00008030EF3201E30F
:101B300089868982896A00008030EF3201E38986D4
:101B40008982896A00008030EF3201E389868982C8
:101B5000896A00008030EF3201E389868982896AD0
:101B600000008030EF3201E389868982896A0000B3
:101B70008030EF3201E389868982896A00008030F3
:101B8000EF3201E389868982896A00008030EE3273
:101B900001E389868982896A00008030EF3201E39F
:101BA00089868982896A00008030EF3201E3898664
:101BB0008982896A00008030EF3201E38986898258
:101BC000896A00008030EF3201E389868982896A60
:101BD00000008030EF3201E389868982896A000043
:101BE0008030EF3201E389868982896A0000803083
:101BF000EF3201E389868982896A00008030EE3203
:101C000001E389868982896A00008030EF3201E32E
:101C100089868982896A00008030EF3201E38986F3
:101C20008982896A00008030EF3201E389868982E7
:101C3000896A00008030EF3201E389868982896AEF
:101C400000008030EF3201E389868982896A0000D2
:101C50008030EF3201E389868982896A0000803012
:101C6000EF3201E389868982896A89848030EE3285
:101C700001E389868982896A89848982899212002E
:101C8000FF0EE3CF1FF0898489828992898489823B
:101C9000896A8982899289828992000080301F3204
:101CA00001E389868982896A000080301F3201E35E
:101CB00089868982896A000080301F3201E3898623
:101CC0008982896A000080301F3201E38986898217
:101CD000896A898480301F3201E389868982896A12
:101CE0008984898289921F50120004011851600B67
:101CF000E842E842E842E842E842000901E0120016
:101D00001951070A4CE00B0A4AE0070A3BE0010AB6
:101D100027E00B0A23E0020A21E0030A1DE0080A7B
:101D200012E0010A0EE00F0A0AE0030A01E01200C5
:101D30000001010EF26F0001040EF96F1200D0EFE6
:101D40000EF035EF0FF00001010EF26F0001FB0EF7
:101D5000F36F000EF46F10D05EEF0FF0A9EF0FF0ED
:101D60000001010EF26F04011C510001F36FF46BCE
:101D7000FC0EF327000EF4230001FA930001010E7C
:101D8000F76F12000001010EF26F04011C51EA6AA4
:101D9000FC0FE96E000EEA221AC4EFFF12001200D7
:101DA000800E0401185D60E11B51030A30E0010A56
:101DB0000CE0030A57E10001010EF26F0001A80ECA
:101DC000F36F270EF46F120E4AD00001010EF26F6E
:101DD00004011A51F66EF76AD890F636F7365C0EA3
:101DE000F626280EF7220900F5CFF3F00A00F5CF0A
:101DF000F4F0020E0001F76AF325F66EF451F722B3
:101E00000900F5CFF7F00A00F5CFF8F02BD000016C
:101E1000010EF26F030E04011A5D0BE18150040BF9
:101E200008E18150080B05E17A0EF66E280EF76E78
:101E30000AD01A51F66EF76AD890F636F736600E69
:101E4000F626280EF7220900F5CFF3F00A00F5CFA9
:101E5000F4F0F3C0F6FFF4C0F7FF0800F5500001FE
:101E6000F76FF86B0001FA8312000001010EF26FA8
:101E70000F0EE66E710EE66E0F0EE66E33EC13F08B
:101E8000E552E552E552010EE66EFC0EE66E000EDE
:101E9000E66E33EC13F0E552E552E5521AC4FBF05E
:101EA00004011A5104E10001050EF96F120000014E
:101EB000060EF96F48EC13F04DEF12F00401206BA1
:101EC000216B040118511F0B020A13E0030A0DE0F5
:101ED000010A31E10001010EF26F040120810001CD
:101EE000FAA129D00401208326D00001010EF26F4F
:101EF00022D00001010EF26F04011C510F0B080DDE
:101F0000F350186A000F176E040E18221C51800B34
:101F100001E0010E040DF35000011724F56F000ECF
:101F20001820F66FF5C0E9FFEA6EEF50040B03E0EE
:101F30000401010E206F0001F2050AE10001200EEC
:101F4000F36F040EF46F0001FA930001020EF76FB5
:101F5000120004011A0510E118511F0B00090CE1D1
:101F60000001010EF26F030E0401195D03E100018F
:101F7000FA8102D00001FA9104011A513AE1185194
:101F80001F0B020836E11C510F0B000932E0000163
:101F9000010EF26F04011C510F0B080DF350186A6B
:101FA000000F176E040E18221C51800B01E0010E69
:101FB000040DF35000011724F56F000E1820F66F82
:101FC000030E0401195D07E1840EF5C0E9FFF6C0B8
:101FD000EAFFEF6E12001CAF06D0F5C0E9FFF6C0B5
:101FE000EAFFEF6A1200880EF5C0E9FFF6C0EAFFCB
:101FF000EF6E12006C5002E0000E01D0010E0009DD
:102000000BE0040100513C0BE842E8420D0802E1FC
:1020100015EF10F027EF10F06C5002E0000E01D029
:10202000010E040901E022D81200D9CFE6FFE1CF6A
:10203000D9FFE6520001F16BF26BF76BF86B75ECB0
:102040000EF0D9D8E552E552E7CFD9FF1200020EC3
:102050000001F15D09E192D8040100BD02D0C80E73
:1020600001D0880E006F120040EF11F0040E000145
:10207000F95D09E11AC46EFF6E50000802E2050E18
:1020800001D0030EF96F0001F10509E10AD804013E
:1020900004BD02D0C80E01D0880E046F120040EFBC
:1020A00011F0D9CFE6FFE1CFD9FF020EE126000102
:1020B000080EF75D000EF85905E2F7C0DEFFF8C024
:1020C000DDFF03D0080EDE6EDD6A04010493049187
:1020D000010EDB500413DFCF05F4000EDB500001CE
:1020E000F75F010EDB50F85B200EF56F040EF66F04
:1020F0000001FAA31DD0D9CFE9FFDACFEAFFEE50F5
:10210000ED1032E0F3C0F6FFF4C0F7FF0800F55021
:10211000F5C0E9FFF6C0EAFFEF6E0001F52B000EF7
:10212000F623F32BF423DF06010EE5E2DB06E3D70B
:10213000D9CFE9FFDACFEAFFEE50ED1015E0F3C09A
:10214000E9FFF4C0EAFFEF50F5C0E9FFF6C0EAFF8F
:10215000EF6E0001F52B000EF623F32BF423DF06C0
:10216000010EE6E2DB06E4D7020EE15C02E2E16A80
:10217000E552E16EE552E7CFD9FF1200D9CFE6FF75
:10218000E1CFD9FF020EE126030E04010015E76E30
:10219000010EE7CFDBFF01C4DFFFDE500001F727B0
:1021A000DD50F823200EF36F040EF46FD9CFE9FF52
:1021B000DACFEAFFEE50ED1014E0F3C0E9FFF4C00F
:1021C000EAFFEF50F5C0E9FFF6C0EAFFEF6EF52B2E
:1021D000000EF623F32BF423DF06010EE7E2DB0605
:1021E000E5D7020EE15C02E2E16AE552E16EE552FA
:1021F000E7CFD9FF12000001F2510BE10401080EF4
:10220000016F180E026F040E036F840E006F04013D
:1022100023D0040118AF22D00001F75104011E5D44
:102220000001F85104011F5904E21EC4F7F01FC455
:10223000F8F037DF0001010EF16F0401080E016FA5
:10224000180E026F040E036F800E006F0401200E43
:10225000066F040E076FC80E046F10D00001020E47
:10226000F16F0401056BC80E046F0401080E016FC5
:10227000200E026F040E036FC80E006F6D981200DF
:102280000001F16B0401080E016F180E026F040EBD
:10229000036F880E006F0401046B12000001A4A1FB
:1022A00070D0040114BF6DD00001A205080DF3CF5A
:1022B000A5F0F4CFA6F0620EA527000EA623A5C0B8
:1022C000E9FFA6C0EAFF020EEB50010A03E0010A93
:1022D00043E057D0A5C0E9FFA6C0EAFF020EE926F9
:1022E000000EEA22020EEF6EA5C0E9FFA6C0EAFFCB
:1022F000040EEB5000091CE0A5C0E9FFA6C0EAFFF0
:10230000040EEB50A26F050EEB50000913E0A5C0C0
:10231000E9FFA6C0EAFF060EE926000EEA22EE0655
:10232000ED5AEECF17F0EDCF18F01750181002E16C
:10233000A49127D0A205080DF3CFA5F0F4CFA6F005
:10234000620EA527000EA623A5C0E9FFA6C0EAFFDE
:10235000020EEB50000915E1A5C0E9FFA6C0EAFF97
:10236000020EE926000EEA22010EEF6EA5C0E9FF7B
:10237000A6C0EAFFEECFE6FFEFCFE6FFBED8E552FC
:10238000E5520001A4A388D0040110BF85D000014C
:10239000A305080DF3CFA5F0F4CFA6F0820EA52774
:1023A000000EA623A5C0E9FFA6C0EAFF020EEB506F
:1023B000010A1BE0010A03E0020A6EE01200A5C058
:1023C000E9FFA6C0EAFF020EE926000EEA22010E8E
:1023D000EF6EA5C0E9FFA6C0EAFFEECFE6FFEFCFA4
:1023E000E6FF77D8E552E5521200A5C0E9FFA6C086
:1023F000EAFF020EE926000EEA22020EEF6EA5C0E9
:10240000E9FFA6C0EAFF040EEB5000091CE0A5C0DE
:10241000E9FFA6C0EAFF040EEB50A36F050EEB50D8
:10242000000913E0A5C0E9FFA6C0EAFF060EE926F1
:10243000000EEA22EE06ED5AEECF17F0EDCF18F0BF
:102440001750181002E1A4931200A305080DF3CF52
:10245000A5F0F4CFA6F0820EA527000EA623A5C0F6
:10246000E9FFA6C0EAFF020EEB50000915E1A5C086
:10247000E9FFA6C0EAFF020EE926000EEA22010EDD
:10248000EF6EA5C0E9FFA6C0EAFFEECFE6FFEFCFF3
:10249000E6FF1FD8E552E5521200D9CFE6FF020E43
:1024A000E1260001606B616B0401480E106F0401AE
:1024B000400E146F1E0E726E0001A491A493020EC2
:1024C000E15C02E2E16AE552E16EE552E7CFD9FF55
:1024D0001200D9CFE6FFE1CFD9FFFD0EDBCF12F41A
:1024E000FE0EDBCF13F40401400E116F1017C80E5F
:1024F000101BE552E7CFD9FF1200D9CFE6FFE1CF9D
:10250000D9FFFD0EDBCF16F4FE0EDBCF17F404016E
:10251000400E156F1417C80E141BE552E7CFD9FFF4
:1025200012006DA60CD80001F90508E16DBA06D0BD
:10253000686A696A69806988020EF96F12006D6ABB
:10254000696A6D860001010EF96F12006D6A696A91
:102550000001F96B1200A6EF12F00001F95101E140
:1025600012006850040B04E06950040B01E038D8F5
:102570006DB212006850010B04E06950010B01E0DC
:1025800050D86850100B04E06950100B01E024D8BB
:102590006850400B04E06950400B01E037D86850A8
:1025A000200B04E06950200B01E032D86850020B88
:1025B00004E06950020B01E032D8030E0001F95D1E
:1025C00001E212006850080B06E06950080B03E0B6
:1025D000FAEC0FF068961200698468986D82120018
:1025E0006D926994689412000001FAA10ED0F8DF90
:1025F0006D840001080EFD6F070EFE6FFD07000ED3
:10260000FE5BFD51FE11FAE16D941200689C120010
:1026100070A003D040EC11F07090689A120068929C
:1026200012006A6A686A9F0E6B6E7B0E696E6E6A34
:102630000F0EE66E710EE66E0F0EE66E14D8E552C2
:10264000E552E552160E706E68A602D06896FCD769
:102650006D9840EC11F00001FA910001FB6B000154
:10266000030EF96F1200D9CFE6FFE1CFD9FFFD0EBF
:10267000DBCFE9FFFE0EDBCFEAFFFC0EDB5004E010
:10268000EE6AFC0EDB06F9D7E552E7CFD9FF120060
:102690000001FF6B1E0E716E0401400E096F280EC3
:1026A0000A6F040E0B6F880E086F0401680E0E6F20
:1026B000040E0F6F400E0C6F1200D9CFE6FFE1CF72
:1026C000D9FFE652FC0EDB50400805E2400EF36EE7
:1026D000FC0EF3CFDBFFDF6AFC0EDB50DF5C19E2A0
:1026E000DF50E76EFD0EDBCFE9FFFE0EDBCFEAFF2A
:1026F000E750E926000EEA22EF50E66EDF50EA6A64
:10270000680FE96E040EEA22E552E750EF6EDF2A09
:10271000E3D7FC0EDBCF0DF4400E04010C17C80EFE
:102720000C1BE552E552E7CFD9FF1200D9CFE6FFE7
:10273000E1CFD9FF0001FF6B040108BF2FD0FC0ED1
:10274000DBCF17F00951D880175403E2FC0E09C4FF
:10275000DBFF0001FF6BFC0EDB50FF5D19E2FF5158
:10276000EA6A280FE96E040EEA22EF50E66EFF5186
:10277000E76EFD0EDBCFE9FFFE0EDBCFEAFFE75091
:10278000E926000EEA22E552E750EF6EFF2BE3D771
:102790000401400E096F0817C80E081B0001FF5105
:1027A000E552E7CFD9FF1200120100020000000835
:1027B000D804E00000000102030109022E0001011B
:1027C0000080FA090400000400000000070501026F
:1027D000400000070581024000000705020240009A
:1027E00000070582024000000403090434034D0081
:1027F0006900630072006F00630068006900700088
:10280000200054006500630068006E006F006C00DB
:102810006F0067007900200049006E0063002E0001
:102820003C03500049004300330032004D00580083
:102830002000530074006100720074006500720093
:1028400020004B0069007400200020002800430095
:10285000290020003200300030003700BA27BA27A4
:10286000E827EC27202800781203300030003000E1
:102870003000300030003000320068282A0EF66E3A
:10288000080EF76E000EF86E00010900F550EC6FAF
:102890000900F550ED6F03E1EC6701D03DD0090070
:1028A000F550E76F0900F550E86F0900F550E96F42
:1028B00009000900F550E96E0900F550EA6E0900BB
:1028C00009000900F550EA6F0900F550EB6F0900A7
:1028D0000900F6CFEEF0F7CFEFF0F8CFF0F0E7C059
:1028E000F6FFE8C0F7FFE9C0F8FF0001EA5302E194
:1028F000EB5307E00900F550EE6EEA07F8E2EB074C
:10290000F9D7EEC0F6FFEFC0F7FFF0C0F8FF000107
:10291000EC07000EED5BBFD712007F000010000037
:102920000000000600000200000040060000030056
:1029300000008006000004000000C0060000000047
:102940000000000700000000000000050200020077
:102950000000400502000101000000050000020027
:102960000000400500000101000004D80FD8CAECA7
:102970000AF0FCD70F0EC112140E6F6E0001F96B36
:102980000001FA6B0001FB6BA3EF0AF091EC12F06F
:102990006FBE02D0ADEC12F0120013EE00F023EE89
:1029A00000F0F86A169C3EEC14F0DBEC14F0B5EC89
:1029B00014F0FBD7120012000000FFFFFFFFFFFF23
:1029C000FFFFFFFFFFFFFFFFFFFFFFFFFFFFFFFF17
:1029D000FFFFFFFFFFFFFFFFFFFFFFFFFFFFFFFF07
:1029E000FFFFFFFFFFFFFFFFFFFFFFFFFFFFFFFFF7
:1029F000FFFFFFFFFFFFFFFFFFFFFFFFFFFFFFFFE7
:0200000400F00A
:020000040030CA
:0E000000210E3F1E000181000FC00FA00F4017
:020000040020DA
:08000000FFFFFFFFFFFFFFFF00
:00000001FF
